:020000040000FA
:02000000F128E5
:0800080004288510851D102855
:10001000051A0B285220851A0E2858201D20052865
:1000200085140030BB2085101F30AB0085190828CF
:100030002B0803190528AB0318280B309F009F18C5
:100040001F281E08F839A700A70CA70CA70C270823
:100050001F39A700A6009320A40008000130A100CA
:10006000C830013C003C031D3128A10B302808009A
:100070005220582052200800851405140C30A80086
:1000800064004720A80B40280510851008002408AC
:10009000A20064000C30A3002E20A30B4C28A20B5E
:1000A000492808006400051447200510472008006F
:1000B000640005140330AC004720AC0B5C2805102D
:1000C00047200800063065280330AC004720AC0B01
:1000D00066280800A9002908A907031D72286420C2
:1000E0001D2000340318762852206B2858206B28D6
:1000F000A50000308A0025088207FC347C343C349B
:100100001C340C3404348434C434E434F4342F0800
:10011000AF0AA50000308A002508820703340034A6
:10012000503400340034A50000308A0025088207CE
:100130006434323421341934143410340E340C3411
:100140000B340A34093408340734073406340634CF
:1001500005340534053405340434043404340434DB
:1001600004340334033403340334033403340334D6
:10017000033402340234AF006400A019C128872080
:10018000C3280008840AA9001D202908003029027C
:10019000031DD028A01DCE28A011BC28A01100341A
:1001A000033029020319DE28013029020319BC2873
:1001B00002302902031DE2286220BC28303084006E
:1001C000A015BC2864002908A907031DE92864209C
:1001D000BC2864000318EE285220E228640058204E
:1001E000E228831285018B010730990009309F00B6
:1001F000831634309F008C01960195010F308100E9
:100200003C30850083121F30AB000330A6009320E2
:10021000A4003830AB00AB032B0883169B001C14E2
:100220001A088312A9002B08303EA5008400290873
:0E0230008000AB08031D0B291C181C29052893
:02400E008C3FE5
:10420000A800D8000200A800D8000200A800D8002A
:10421000020090004000020048003000C400080086
:10422000C800020048003000C4000800C8000200B6
:1042300048003000C4000800C8000200B0000000C0
:04424000000000007A
:00000001FF
